:100000000C9496010C94BE010C94BE010C94BE019C
:100010000C94BE010C94BE010C94BE010C94BE0164
:100020000C94BE010C9437030C94EA230C949C228C
:100030000C94BE010C94BE010C94BE010C94BE0144
:100040000C94540A0C94BE010C94BE010C94BE0195
:100050000C94BE010C94BE010C94BE010C94B81A11
:100060000C94BE010C94911F0C94D41F0C94BE01EF
:100070000C94BE010C94BE010C94BE010C94BE0104
:100080000C94BE010C94BE010C94BE010C94BE01F4
:100090000C94BE010C94BE010C94BE010C94BE01E4
:1000A0000C94BE010C94BE010C94BE012B133113B1
:1000B00037133E134C136E138C13C11BC41BB71B99
:1000C000BB1BE51BE51BE51BC81BCC1BD01BD61BB4
:1000D000DA1BE51BE01B434C49206E6F74206176F0
:1000E00061696C61626C652C2075736520636F6E4D
:1000F000666967757261746F72210000000002000A
:10010000080E0000030401000B00000000000000C6
:100110000000000000000000000408020110408000
:1001200040102040804080080204018040201002DE
:10013000011080102040400404040404030405025C
:100140000202020403020202020606060606060472
:100150000402020204000000002300260029002CF3
:10016000002F0000000000250028002B002E003189
:100170000000000000240027002A002D00300008A5
:100180000B0002020201000904000001020200004B
:1001900005240010010524010101042402060524A0
:1001A0000600010705810310004009040100020A4E
:1001B000000000070502024000000705830240001E
:1001C0000000C18081C112010002020000404123F1
:1001D000368000010102000112010002000000400F
:1001E0004123368000010102000118034100720022
:1001F0006400750069006E006F0020004C004C0028
:1002000043002203410072006400750069006E0023
:100210006F0020004C0065006F006E0061007200EE
:1002200064006F00040309040000000000000000E7
:100230002A2B280000000000000000000000000041
:1002400000000000000000002C9EB4A0A1A2A43475
:10025000A6A7A5AE362D3738271E1F20212223241E
:100260002526B333B62EB7B89F8485868788898ABA
:100270008B8C8D8E8F909192939495969798999A56
:100280009B9C9D2F3130A3AD350405060708090A54
:100290000B0C0D0E0F101112131415161718191A36
:1002A0001B1C1DAFB1B0B500090402000103000022
:1002B00000092101010001226500070584034000B7
:1002C0000105010902A1010901A100850105091922
:1002D000012903150025019503750181029501751A
:1002E00005810305010930093109381581257F751C
:1002F0000895038106C0C005010906A10185020514
:100300000719E029E7150025017501950881029577
:1003100001750881039506750815002565050719FF
:100320000029658100C0721DC220862511241FBED0
:10033000CFEFDAE0DEBFCDBF12E0A0E0B1E0E8EB46
:10034000FDE402C005900D92AA35B107D9F715E07A
:10035000AAE5B2E001C01D92AC31B107E1F713E0AC
:10036000CCE2D3E004C02297FE010E944F26C632A1
:10037000D107C9F70E94FE200C94DA260C940000E5
:1003800080910008909101088737974709F0A89558
:100390000895DC01ED91FC910190F081E02D09952B
:1003A00008952091A0033091A103382748E0C901A6
:1003B000880F991F37FF06C09C0151E2252750E1A5
:1003C000352701C09C01415091F73093A103209340
:1003D000A003089588E38093A20380E092ECA1E05B
:1003E000B0E08093A3039093A403A093A503B093DC
:1003F000A60387E08093AF0380EC9AECA9E8B6E30C
:100400008093A7039093A803A093A903B093AA0392
:1004100085E08093B0038DEE9EEFADEABEED809354
:10042000AB039093AC03A093AD03B093AE03E1EBA9
:10043000F3E080E090E0863028F4DC01AC5DBD4F55
:100440002C9101C020E0219301968831910599F704
:1004500082E08093C9038AE08093CA03089580EC08
:1004600097EFAAEBB7E38093E7039093E803A09399
:10047000E903B093EA0380E090E0A0E0B0E5809368
:10048000EB039093EC03A093ED03B093EE03EFEE38
:10049000F3E080E081938F5F8031E1F70895A0E081
:1004A000B0E0E5E5F2E00C941826D82F0E940E1B70
:1004B0006115710581059105C9F30E94BB26109253
:1004C000AB031092AC031092AD031092AE03C4E0E4
:1004D000812C912C54018A94C090AB03D090AC0332
:1004E000E090AD03F090AE03FE2CED2CDC2CCC2480
:1004F0000E94B626A50194010E94F7256C0D7D1D72
:100500008E1D9F1D6093AB037093AC038093AD036E
:100510009093AE03C15001F7DD2309F450C001EB05
:1005200013E0E801A12CB12C62E3C62ED12CE12C02
:10053000F12C8881882309F442C0B39419F40E94F5
:10054000EA013DC00E94B626A70196010E94F72548
:10055000E1E0E60FA1EBB3E08A2F801B8A1520F4BF
:100560008D918E13F9CFE9CF2091B00330E0A0E157
:10057000B7E20E948F259B01AC01AE2FB0E00E9434
:100580009E254090A7035090A8036090A903709007
:10059000AA03640D751D861D971D4090E7035090BA
:1005A000E8036090E9037090EA0346165706680670
:1005B000790618F2E993A39488E1A812BACFCDB7CF
:1005C000DEB7E0E10C94342680919F03813019F46A
:1005D00082E080939F0380919F03833019F484E02D
:1005E00080939F03089588E08093C10061E08AE0D2
:1005F0000E94E61B60E08AE00E941F1C089500979D
:10060000C9F09C0140E050E068E478EE81E090E0C1
:100610000E94F7252F3F31054105510529F020F0B3
:100620002FEF30E040E050E02093D1008091C000F7
:10063000806103C08091C0008F7E8093C0000895C8
:10064000219A229A239860E08BE00E94E61B61E0E9
:100650008CE00E94E61B0895EBE6F0E08081806864
:100660008083E8E6F0E080818160808308951F92B6
:100670000F920FB60F9211242F933F934F935F93D6
:100680006F937F938F939F93AF93BF93EF93FF935A
:100690001F9B0E94E402FF91EF91BF91AF919F9148
:1006A0008F917F916F915F914F913F912F910F901B
:1006B0000FBE0F901F901895A1E0B0E0E2E6F3E0C6
:1006C0000C9425261FB791E090939E03F89489839C
:1006D0000E94C00198E1909360008981809360003E
:1006E00081110E94C0011FBF2196E3E00C944126B6
:1006F0008F929F92AF92BF92CF92DF92EF92FF9232
:10070000CF93FC01C0A5EC2FE770F0E0E45EFD4F55
:10071000A081B0E0C7FF03C024E130E002C02FE0B9
:1007200030E0FC0197A183E1989FF0011124E25C85
:10073000FE4F80809180A280B380A20FB31F20E47F
:100740003FE14DE750E00E94A925A50194010E94D8
:10075000D5258C2F887149F469017A01E0EDCE0E20
:10076000E7E0DE1EE11CF11C1BC0C7FF05C060E412
:100770007AE88CE29EE004C060E07EEE8AEB9BE0CB
:1007800069017A01F8EBCF0EFBE0DF1EE11CF11CE2
:10079000A50194010E94D525C20ED31EE41EF51EAC
:1007A000C701B60169517C4F8F4F9F4F28EE33E050
:1007B00040E050E00E94D525A8EEB3E00E949E25BF
:1007C000CF91FF90EF90DF90CF90BF90AF909F9030
:1007D0008F9008958F3F910551F048F0811522E0E8
:1007E000920738F08115934030F482E0089580E05C
:1007F000089581E0089583E00895A0E0B0E0E3E08B
:10080000F4E00C942126EB018A01B82FB695A0E004
:1008100028813981F80120832A813B8121832C8121
:100820003D8122832E813F812383688179814A81A2
:100830005B812C813D81EE81FF819F2F9295990FE5
:10084000990F907C272F2370922B252F2370220F36
:10085000220F922B232F23702295207F922BF801B9
:1008600094830B5F1F4F2896AF5FBA1788F680FFFF
:1008700024C0888199810E94EA03D82E8A819B81B5
:100880000E94EA03E82E8C819D810E94EA03F82EE3
:100890008E819F810E94EA03F0E4DF9EA001112473
:1008A00090E1E99E90011124242B282BE4E0FE9E88
:1008B000B0011124262BF8012083CDB7DEB7E7E085
:1008C0000C943D26803223E0920708F1883E23E015
:1008D000920740F48F519340E4E096958795EA950E
:1008E000E1F70895803D27E0920718F48C5D93406E
:1008F0000895883928E0920768F4885C974074E08E
:10090000969587957A95E1F78D509C4F089580E0F4
:1009100090E008958FEF93E008958C30910540F4B6
:10092000A4E0880F991FAA95E1F7885D9C4F089570
:10093000843F23E0920718F484529C4F0895811558
:1009400024E0920740F48657934FF4E0880F991FF4
:10095000FA95E1F7089580E998E008959C013695AD
:10096000279525753575821B930B9C012373337373
:10097000969587959695879583739373820F931FAA
:100980009C0154E0369527955A95E1F7280F391FB9
:100990002F703F7041E051E0249FC001259F900DD2
:1009A000349F900D1124892F08952998882319F0D8
:1009B00000002A9A02C000002A980000299A00002C
:1009C0000895299A000083B12998000083FB8827A5
:1009D00080F90895CF93DF93D82F5E9A29985E9877
:1009E000C8E08D2F80780E94D504DD0FC150C9F773
:1009F0002998DF91CF9108958F770E94EA04089596
:100A0000CF93DF93D82FC8E08D2F80780E94D50434
:100A1000DD0FC150C9F72998DF91CF910895CF9389
:100A2000DF932998C8E080E0D82FDD0F0E94E10411
:100A30008D0FC150C9F7DF91CF9108950E94FC043A
:100A40000E940F055E9A0895A1E0B0E0EAE2F5E0A9
:100A50000C942626806869830E94EA046981862FA7
:100A60000E9400055E9A2196E2E00C944226CF9304
:100A7000C091AB03C827E82FF0E0EE55FC4F678527
:100A800089E70E9424056C2F8DE30E9424056C2FBA
:100A900082E40E942405CF91089586E20E941E05FB
:100AA0000895CF93DF93EC016C818CE10E942405C3
:100AB0006D818DE10E9424056E818EE10E942405E6
:100AC0006F8180E20E942405688581E20E942405EE
:100AD000698582E20E9424056A8583E20E942405DA
:100AE0006B8584E20E9424056C8585E20E942405C2
:100AF0006D858AE20E9424056E858EE60E9424059B
:100B00006F858FE60E942405688980E70E9424058E
:100B1000698981E70E9424056A8982E70E94240589
:100B2000DF91CF910895CF92DF92EF92FF92CF9312
:100B3000DF936B017C01C11488E3D8068CE9E806D9
:100B40008CE1F80628F5C701B60120E836E948E946
:100B500050E00E94D525E901689760E879E687E6CC
:100B60009FEF0E94B1256C0D7D1D8E1D9F1DF2E033
:100B7000660F771F881F991FFA95D1F721E732E09A
:100B800040E050E00E94D525F22EE32E80E421C003
:100B9000C701B60120E03DE241E351E00E94D525C6
:100BA000E901689760E073ED8EEC9EEF0E94B1253D
:100BB0006C0D7D1D8E1D9F1D660F771F881F991F51
:100BC00021E732E040E050E00E94D525F22EE32EEE
:100BD00080E66C2F6F71680F85E70E9424056E2DEB
:100BE00086E70E9424056F2D87E70E942405DF9188
:100BF000CF91FF90EF90DF90CF900895682F8DE612
:100C00000E94240508958F929F92AF92BF92CF9237
:100C1000DF92EF92FF92CF93DF93D82F83E00E9471
:100C20001E0580939D0384E00E941E0580939C0313
:100C300060E086E00E94240561E087E00E942405D0
:100C40006FE789E00E94240565E08AE00E942405A0
:100C500065E18BE00E94240562E18CE00E9424059E
:100C60006DEF8DE00E94240560E08EE00E94240577
:100C7000DD2319F08BE291E008C02091C90333E134
:100C8000239FC0011124825C9E4F0E9451056CE895
:100C900080E30E9424056FE082E30E94240562E461
:100CA00083E30E9424058091CA0387FF02C064E1A8
:100CB00001C06AE084E30E9424056AE285E30E94A1
:100CC00024056DE286E30E94240564ED87E30E941B
:100CD000240560E088E30E94240560E089E30E9427
:100CE0002405D11109C0C090AB03D090AC03E090B3
:100CF000AD03F090AE0307C0C5E9CC2EC1ECDC2EED
:100D0000ED2CCEEDFC2ECAE38F2C9924AA24BB2413
:100D1000682D8C2F0E942405682D85E08C0F0E9481
:100D20002405FE2CED2CDC2CCC24CF5FCE3361F7D8
:100D30006FEF83E40E9424056FEF84E40E94240592
:100D40006FEF85E40E9424056FEF86E40E9424057E
:100D5000DD2311F066E002C06091AF038DE60E94D2
:100D6000240560E089E70E9424056091B0038AE7CA
:100D70000E94240560E083E70E94240560E084E788
:100D80000E942405D11109C06091A7037091A803A6
:100D90008091A9039091AA0304C060EC7AEC89E8E1
:100DA00096E30E949305DF91CF91FF90EF90DF9043
:100DB000CF90BF90AF909F908F90089561E087E0B3
:100DC0000E94240564E28EE70E94240563E088E027
:100DD0000E94240560E088E00E94240565E087E029
:100DE0000E94240562E085E00E94240583E00E94C1
:100DF0001E0580939D0384E00E941E0580939C0342
:100E0000089583E00E941E0580939D0384E00E9464
:100E10001E0580939C0361E087E00E9424056AE040
:100E200070E080E090E00E94311B0E94DE0600002E
:100E30000895CF92DF92FF920F931F93CF93DF938A
:100E40001F92CDB7DEB7082F162F8EE399830E942D
:100E50002405F02EC02E9981D92E8C2D8F19811743
:100E600038F4F60161916F018FE70E942405F5CFF8
:100E700064E085E00E94240583E00E941E058093C3
:100E80009D0384E00E941E0580939C030E940E1B1C
:100E9000609398037093990380939A0390939B03B4
:100EA00069E087E00E94240581E080939F030F9012
:100EB000DF91CF911F910F91FF90DF90CF90089518
:100EC0000F931F930E94190780919F03813099F41B
:100ED0000E940E1B009198031091990320919A0390
:100EE00030919B03601B710B820B930B603A764829
:100EF0008140910548F380919F03813031F467EA86
:100F000071E08AE094E00E94161E1F910F910895EF
:100F10000F931F9380919F03823021F410929F03BF
:100F200081E020C080919F038130D9F40E940E1B84
:100F3000009198031091990320919A0330919B039B
:100F4000601B710B820B930B613A764881409105CF
:100F500040F061E087E00E94240510929F0382E048
:100F600001C080E01F910F910895CF93DF93EC01B2
:100F70004AE050E06D2F70E08AE094E00E94DB1EB2
:100F80006EE28AE094E00E94E81DBE0184E076955E
:100F900067958A95E1F76F7077274AE050E08AE01D
:100FA00094E00E94DB1E6EE28AE094E00E94E81D5D
:100FB000BE016F7077274AE050E08AE094E00E941B
:100FC000DB1EDF91CF910895D82FC0E0CD1780F4BC
:100FD0005F9A64E670E080E090E00E94311B5F98C9
:100FE00064E670E080E090E00E94311BCF5FEECFBE
:100FF0006CE271E080E090E00E94311BE6CF0F933D
:101000001F93CF93DF93EC01062F15E0115051F0A1
:10101000CE010E94C426081741F0602FCE010E9425
:10102000CC26F4CF82E00E94E407DF91CF911F919C
:101030000F910895A0E0B0E0E0E2F8E00C941826EB
:10104000482E562EC0E0D0E0612C712CE12CF12C02
:1010500000E010E041100CC06090000486E4689E3F
:101060003001112459E1E52EF12C06EE13E01EC0EB
:1010700091E049120FC060900004E6E46E9E3001DA
:101080001124FBE16F0E711C49E2E42EF12C02EAFF
:1010900013E00CC082E0481209C028E1622E7724D8
:1010A0007394EE24E394F12C0FEF13E043018C0EC4
:1010B0009D1E1092A1031092A0033401A62CA81823
:1010C000B12CC30101966C01AE14BF04A8F4A00EAC
:1010D000B11E511006C0C3010E94C426F5018083D1
:1010E00005C0F5016081C3010E94FF07F501808101
:1010F0000E94D1013601E2CFC301511018C0C301D3
:101100000E94C426B82EC6010E94C4262B2D30E0B2
:10111000322F2227282B8091A0039091A1038217C0
:10112000930779F4C0E0D0E05524539493CF36016F
:101130006091A1030E94FF076091A003C6010E9475
:10114000FF07C05EDE4FC13E92E0D90708F482CFB0
:10115000852DCDB7DEB7E0E10C94342661E082E066
:101160000E941A08089560E082E00E941A088091A7
:10117000FF03853020F01092FF030E94AE0880919B
:10118000FF0380930004089561E080E00E941A0844
:1011900061E081E00E941A08089560E080E00E940A
:1011A0001A08882351F060E081E00E941A08882321
:1011B00021F08091A203883349F00E942F020E94FF
:1011C000EA0181E00E944F020E94C4080895CF9373
:1011D000C82F0E940E1B60935C0370935D03809385
:1011E0005E0390935F03C0937103CC2329F040E02A
:1011F00051EE60E070E004C040E855E260E070E06D
:101200008CE594E00E944120CF9108959091600375
:10121000492F4F7050E0BA016F5F7F4F292F30E0A8
:10122000E4E035952795EA95E1F76217730759F0E1
:10123000FA01EF59FC4F808381E0890F8F70907F16
:10124000892B8093600308956EE770E08CE594E04D
:101250000E94C9010895A3E1B1E0E1E3F9E00C9433
:101260001926E1EBF3E0712C8191882321F073942E
:1012700028E17212F9CF63EB71E08AE094E00E94FA
:10128000161E4AE050E0672D8AE094E00E94E21EBC
:1012900080E00E9403060E94DE068E010E5F1F4F53
:1012A000C12CD12C7601C39466246A945C2C0E94D4
:1012B000021B4B015C012091B00330E0A0E1B7E2DA
:1012C0000E948F259B01AC01C701B6010E94B12588
:1012D0002091A7033091A8034091A9035091AA033C
:1012E000620F731F841F951F2091E7033091E8035D
:1012F0004091E9035091EA03261737074807590739
:1013000018F4F801608225C08C2D0E94370561E039
:1013100070E080E090E00E94311BF80110820E9492
:10132000021B681979098A099B09643F714081058C
:10133000910540F40E944D05F8019081981778F7C7
:101340008083EDCF50FE03C046985F9A02C0469A54
:101350005F982FEFC21AD20AE20AF20A0F5F1F4FFC
:101360008FEFC816D104E104F10409F09FCFCE013C
:101370009395FC01D82E7FEF68EC2E2F281B2715A4
:1013800010F051E056C0DE01129651E02FEF41E01F
:101390003D91321710F0322F01C0452F5F5F5F3F44
:1013A00011F0232FF5CF4193242F30E0A1E0B0E0DE
:1013B000AC0FBD1FA20FB31F5C93413079F0DE016B
:1013C000A20FB31F5C93423049F0AFEFBFEFAC0FF9
:1013D000BD1FA20FB31F6C934E3F78F6A2E0B0E0A2
:1013E000AC0FBD1FA20FB31F7C934D3F30F6A3E09F
:1013F000B0E0AC0FBD1FA20FB31F6C93BECF452F43
:10140000242F30E0FC01E20FF31F6081AFEFB0E06A
:10141000AC0FBD1FA20FB31F2C91621748F44150AF
:10142000DC01A40FB11D2C9120836C934111E8CFF6
:101430005F5F571520F3372D369520E0231770F4A2
:10144000DC01A20FB11D4C91522F530FFC01E50F8F
:10145000F11D50815C9340832E5FF0CFF1EBEF2EB6
:10146000F3E0FF2E8C01802F8D19871598F4F80179
:10147000C1908F014AE050E06C2D8AE094E00E9418
:10148000D31E6CE28AE094E00E94E81DF701C1924D
:101490007F01E9CF8AE094E00E94F01D81E0CD5EFB
:1014A000DE4FEFE00C9435261F920F920FB60F928D
:1014B00011241F932F933F934F935F936F937F93C9
:1014C0008F939F93AF93BF93CF93DF93EF93FF934C
:1014D000C0918600D09187008091170390911803E6
:1014E00020913903211155C09E01281B390B809191
:1014F000EB039091EC03A091ED03B091EE0385FD19
:1015000002C036952795253C49E03407B8F1409153
:101510000A0150E060E070E02CE1B695A795979540
:1015200087952A95D1F70097A105B10521F481E0AF
:1015300090E0A0E0B0E084179507A607B707D8F4BD
:1015400080910A018F3FB9F040E080910A0148176D
:1015500080F4842F90E0880F991FFC01E75EFC4F18
:1015600020813181FC01E55FFE4F318320834F5F95
:10157000ECCF10923A0310920A010BC02D3B82E08F
:10158000380720F080910A018031D8F08FEF8093E6
:101590000A01D0931803C0931703FF91EF91DF91D5
:1015A000CF91BF91AF919F918F917F916F915F91FB
:1015B0004F913F912F911F910F900FBE0F901F9051
:1015C000189510910A0181E0810F80930A01C901E9
:1015D0000E946204E12FF0E0EE0FFF1FE75EFC4F78
:1015E00091838083D6CF83E0809380008AE98093C3
:1015F00081008091EB0386FD05C0809181008064AD
:10160000809381008FEF9FEF9093890080938800F3
:1016100080916F00806280936F000895CF93DF9375
:101620000E94B30880910004843039F582E00E9462
:10163000521CC1E0D0E0892B11F4C0E0D0E083E07F
:101640000E94521C892B19F082E090E002C080E0D9
:1016500090E08C2B9D2B8230910539F083309105E1
:1016600039F0019739F481E006C01092000405C0FA
:1016700082E001C083E080930004DF91CF91089560
:101680006F3018F086958058089589E0689F802D06
:1016900011240895A0E0B0E0E0E5FBE00C942026E2
:1016A000C82F0E940E1B0091C8021091C902209100
:1016B000CA023091CB026B017C01C01AD10AE20A46
:1016C000F30A9701860149E8C41643E1D406E10410
:1016D000F10410F01092CC026093C8027093C9021A
:1016E0008093CA029093CB02209139038FEF820F2F
:1016F0008230E8F5E091CC02EE2309F46EC1E130CE
:1017000011F482E0D8C1E03178F581E08E0F80934A
:10171000CC02F0E0E75EFC4FC083803109F0D4C119
:10172000EBE1F3E0213029F4A181A695A695808113
:1017300008C080819181A92FA695A695A69596951A
:101740008795A03148F4B0E090E0AA0FBB1FA55FD9
:10175000BE4F11969C938E9310923A03329683E07B
:10176000E932F807F9F6B0C11092CC02ADC12330CE
:1017700009F023C1E091CC02E11118C0CF3009F08B
:1017800011C10E94021B0091470310914803209150
:10179000490330914A03601B710B820B930B62303B
:1017A00071058105910508F089C1FCC0E73148F455
:1017B00081E08E0F8093CC02F0E0E85EFC4FC083A6
:1017C000F1C0E73109F0ECC0C111EAC040E050E0DF
:1017D000ABE0CA01B3E0880F991FBA95E1F7A49F67
:1017E0009001A59F300D1124F901E75EFC4F608147
:1017F000E1817E2F777075956795FC01EE0FFF1FD5
:10180000E55FFE4F71836083F901E65EFC4FB081B6
:10181000B695B695B695E181FE2FF295FF0FF07E55
:101820006F2F6B2BE695E695E6957E2F7770759575
:101830006795FC01EE0FFF1FE35FFE4F718360832E
:10184000F901E55EFC4FB081B295B695B695B370DF
:10185000C181DC2FDD0FDD0F6D2F6B2BC295C6957F
:10186000C695C370E281E170EE0FEE0F7E2F7C2BE8
:1018700075956795FC01EE0FFF1FE15FFE4F7183C9
:101880006083F901E35EFC4FB081B695E181FE2FE4
:10189000F795FF27F7956F2F6B2BE6957E2F7770C7
:1018A00075956795FC01EE0FFF1FEF5EFE4F71838C
:1018B0006083F901E25EFC4FB081B295BF70E181B7
:1018C000FE2FF295F07F6F2F6B2BE295EF707E2F3E
:1018D000777075956795FC01EE0FFF1FED5EFE4F6B
:1018E00071836083F901E15EFC4FB081BB1FBB27B0
:1018F000BB1FC181DC2FDD0F6D2F6B2BCC1FCC27C5
:10190000CC1FE281E370EE0F7E2F7C2B75956795DF
:10191000FC01EE0FFF1FEB5EFE4F71836083F90148
:10192000EF5DFC4FB081B695B695E181FE2FF29543
:10193000FF0FFF0FF07C6F2F6B2BE695E6957E2F48
:10194000777075956795FC01EE0FFF1FE95EFE4FFE
:1019500071836083F901EE5DFC4F2081229526950D
:1019600027703181E32FEE0FEE0FEE0F6E2F622BFB
:10197000732F72957695777075956795FC01EE0FCC
:10198000FF1FE75EFE4F718360834F5F5F4F423002
:10199000510509F01ECF80912F0383FF10923A0367
:1019A0001092CC020E94021B60934703709348037D
:1019B0008093490390934A0387C0243009F084C080
:1019C0006091CC0261110BC0C83AB1F41092A1032E
:1019D0001092A00388EA0E94D10181E06CC06130BE
:1019E00019F4C093C70204C0623031F4C093C60238
:1019F0008C2F0E94D1015AC0E091C6022E2F30E0F8
:101A0000220F331F462F50E0C90102968417950715
:101A10003CF0633268F7FA01EA5EFC4FC083E8CF1E
:101A20002D5F3F4F8C2F90E06091A0037091A10338
:101A30004217530749F4982F8827862797279093B2
:101A4000A1038093A00332C06817790769F58091DC
:101A5000C702813049F5E13118F080E18093C60278
:101A6000F090C602CAE1D3E000E010E00F15D0F418
:101A7000FE013197808190E0982F88272881822B62
:101A800063E0969587956A95E1F70E946204F801F4
:101A9000EE0FFF1FE55FFE4F918380830F5F1F4FA7
:101AA0002296E4CF10923A031092CC028091CC029D
:101AB000882351F08F5F8093CC0206C08091CC02C6
:101AC0008F5F8093CC026ECFCDB7DEB7E8E00C9489
:101AD0003C26CF93DF93E82FF0E0EA51FC4FE185FD
:101AE000E03150F4F894F0E0EE0FFF1FE55FFE4F99
:101AF0008081918178945FC08EE08E0F8B3058F496
:101B0000F0E0E25FF10924E62E9FC0012F9F900DC7
:101B100011240C9650C0E03F09F448C038F4E1317C
:101B2000A1F0E231A1F0E03139F409C0ED3FC1F19B
:101B3000EE3FC9F1E13F89F180E092E03CC082E0F4
:101B40000E94521C892B19F134C083E0F9CF82E046
:101B50000E94521CC1E0D0E0892B11F4C0E0D0E01B
:101B600083E00E94521C892B19F082E090E002C0B1
:101B700080E090E08C2B9D2B8230910541F08330EA
:101B8000910541F00197A9F086EA92E014C08CE03B
:101B900090E011C089E591E00EC086E090E00BC0B6
:101BA0008AEF93E008C08FEF93E005C080E090E0FB
:101BB00002C084EF93E0DF91CF910895A2E2B0E0FC
:101BC000E4EEFDE00C9416269E012F5F3F4F80E16E
:101BD000D9011D928A95E9F761EE71E08AE094E0FF
:101BE00029A33AA30E94161E0E9401071D8A1E8A7D
:101BF0001F8A188E312C212C00E0812C912C54014D
:101C000070EC472E7DE9572E78E5672E75E3772E29
:101C1000E0E5CE2EE3ECDE2EE12CF12C84EF91E01A
:101C2000A0E0B0E08D8F9E8FAF8FB8A380EC97EFD0
:101C3000AAEBB7E3898F9A8FAB8FBC8F80EC9DE9BD
:101C4000A8E5B5E3898B9A8BAB8BBC8B8AE094E0DB
:101C50000E947B1C892B09F4E1C08AE094E00E9479
:101C60009F1C9C0133272C32310509F442C0ACF48F
:101C70002332310509F0ABC019821A821B821C8203
:101C80001D821E821F82188619861A861B861C8654
:101C90001D861E861F86188A60C02434310529F0EF
:101CA0002335310509F4B2C092C064E48AE094E0BF
:101CB0000E94E81D2AE030E040EC5DE968E575E34C
:101CC0008AE094E00E94761E6CE28AE094E00E9432
:101CD000E81D2AE030E040EC57EF6AEB77E38AE05A
:101CE00094E00E94761E6CE28AE094E00E94281E36
:101CF000ADCF0F5F043009F0A9CF29813A814B8124
:101D00005C81A8EEB3E00E949E25698B7A8B8B8B59
:101D10009C8B2D813E814F8158850E949E25698F25
:101D20007A8F8B8F9C8F29853A854B855C852D8F8B
:101D30003E8F4F8F58A32D853E854F8558890E9431
:101D40009E256B017C0160323EE47307810591059D
:101D500030F462E38CE10E94240500E077CF603329
:101D600045E774078105910510F462E2F3CF603412
:101D70005CE975078105910510F466E2EBCF80E51B
:101D8000C81683ECD806E104F10410F462E1E2CF56
:101D900090E6C9169AEED906E104F10410F465E163
:101DA000D9CFA0E7CA16A1E1DA06A1E0EA06F1045C
:101DB00010F461E0CFCFB0EACB16B6E8DB06B1E0B5
:101DC000EB06F10410F463E0C5CF65E0C3CF10ED7E
:101DD000180F1A3008F03ACFE1E0F0E0EC0FFD1FE9
:101DE00024E0029FE00DF11D112420813181428108
:101DF0005381AAE0B0E00E949E25610F711D811DF4
:101E0000911D608371838283938320CF49885A8890
:101E10006B887C88812C912C540118CF81149104FB
:101E2000A104B10489F4C301B2010E94930561E0E9
:101E300070E080E090E00E94311B1D8A1E8A1F8A9C
:101E4000188E312C22242A948D8D9E8DAF8DB8A1B1
:101E500088169906AA06BB06D0F40E944D052D8966
:101E60003E894F89588D280F311D411D511D2D8BE5
:101E70003E8B4F8B588F381608F4382E821508F495
:101E8000282E3FEF831A930AA30AB30A56C0C30150
:101E9000B20128EE33E040E050E00E94D525BA01BF
:101EA000A9012AE030E08AE094E00E94C41E6CE2BE
:101EB0008AE094E00E94E81D4AE050E0632D8AE049
:101EC00094E00E94D31E6CE28AE094E00E94E81D38
:101ED0006D897E898F89988DA50194010E94D525F1
:101EE000BA01A9012AE030E08AE094E00E94C41E11
:101EF0006CE28AE094E00E94E81D4AE050E0622D26
:101F00008AE094E00E94D31E6CE28AE094E00E9492
:101F1000281E4C0C5D1C6E1C7F1C898D9A8DAB8D10
:101F2000BC8D84159505A605B70520F449885A8807
:101F30006B887C88812C912C540129893A894B89A2
:101F40005C89283E33404105510509F07FCEA296B9
:101F5000E2E10C943226ACE1B0E0E1EBFFE00C945E
:101F600020260E940E1B6B017C0181E00E9403066B
:101F700014E703E0198361E0CE0101960E94600737
:101F800000939F030E94DE066AEF70E080E090E01D
:101F90000E94311B80919F03833089F48AE094E092
:101FA0000E947B1C892B59F40E940E1B6C197D0921
:101FB0008E099F096038734C894C9140D8F280910A
:101FC0009F03833009F44FC08FE70E94FC040E94F6
:101FD0000F058983843511F083E05CC00E940F05F2
:101FE00010927203809373030E940F052091720375
:101FF00030917303280F311D3093730320937203C4
:102000000E940F05809374030E940F05809375034F
:10201000813110F7F12C0F2D10E08091750390E0C5
:10202000880F991F0817190740F40E940F05F8013F
:10203000EA58FC4F8083F394EECF80E7898361E018
:10204000CE0101960E94600783E080939F030E9467
:10205000DE0662E370E080E090E00E94311B809138
:102060009F03833011F482E015C08FE70E94FC04C7
:102070000E940F058983803509F0AECF0BEC13E089
:102080000E940F05F80181938F01F3E0063E1F07C0
:10209000B9F781E06C96E8E00C943C26CF93C82F0A
:1020A000682F8AE094E00E94EC1C909196039C2794
:1020B00090939603CF910895A1E0B0E0E2E6F0E1BD
:1020C0000C94262699830E944E109981892F0E9494
:1020D0004E102196E2E00C9442261F93CF93DF939B
:1020E000182FEB011092960365EB8AE094E00E94B2
:1020F000EC1C62E68AE094E00E94EC1C812F0E94B6
:102100004E10CE010E945C10DF91CF911F91089577
:10211000609196038AE094E00E94EC1C0895A1E28D
:10212000B0E0E5E9F0E10C9422267B018A018C30D5
:1021300009F453C108F040C0863009F4BCC018F55A
:10214000833009F491C070F4813009F472C0823098
:1021500009F048C26BE170E082E00E946D100BEC68
:1021600013E078C0843009F487C0853009F03AC2A2
:102170006091750370E0660F771F85E00E946D1017
:1021800006E713E086C0893009F4A7C070F48730F1
:1021900009F49BC0883009F025C261E070E088E056
:1021A0000E946D108091000423C28A3009F4CAC0D5
:1021B0008B3009F4F2C016C28A3609F475C1D8F41E
:1021C000873609F43AC138F4853609F40EC18636EB
:1021D00009F41FC107C2883609F437C1893609F0EE
:1021E00001C261E070E089E60E946D100E94EA0180
:1021F0000E942F02F5C18D3609F4D4C138F48B3614
:1022000009F491C18C3609F49AC1ECC18E3609F4F7
:10221000DCC1873C09F0E6C161E070E087EC0E9418
:102220006D1081E00E944E100E948810109297035A
:10223000E3C169E270E081E00E946D1002EA13E000
:10224000F80181918F010E944E10F3E00B3C1F07B3
:10225000B9F7D0C1F80181918F010E944E10F3E0CF
:10226000063E1F07B9F7C6C161E070E083E00E9437
:102270006D100E94AB0FBCC161E070E084E00E9471
:102280006D1081E00E944E100E9488100E94DE0DA9
:10229000B3C18091750390E0880F991F980126576C
:1022A00033402817390708F0A5C1F80181918F0143
:1022B0000E944E10EECF62E070E086E00E946D104A
:1022C00086E893E00E945C1095C161E070E087E0D1
:1022D0000E946D10809174038BC186E6898361E052
:1022E000CE0101960E9460070E94DE0683E0809383
:1022F0009F0368EC70E080E090E00E94311B8091C9
:102300009F038430D9F48FE70E94FC040E940F05DC
:102310008983863469F460E270E089E00E946D1080
:1023200010E20E940F050E944E101150D1F762C1B9
:1023300061E070E089E00E946D1052C161E070E0E0
:1023400089E053C169E170E08AE00E946D1082E08B
:102350008093E60320919E038091EB039091EC0320
:10236000A091ED03B091EE03222311F0806801C02B
:102370008F778093EB039093EC03A093ED03B093DE
:10238000EE0306EE13E0F80181918F010E944E10DA
:10239000F3E00F3F1F07B9F72DC161E270E08BE05A
:1023A0000E946D1080913A038F3F39F080913A037B
:1023B00091E0980F90933A0302C080913A030E94F3
:1023C0004E1010E0812F0E94690D0E948D040E9422
:1023D0005C101F5F1031B1F70DC161E070E08CE05F
:1023E0000E946D108091FF0303C161E070E085E6FB
:1023F0000E946D1089E2E816F10409F0F8C0D801D6
:10240000E2EAF3E08D91819383E0EB3CF807D1F7AA
:10241000E7C061E070E086E60E946D10EBE1EE1629
:10242000F10409F0E4C0D801EBECF3E08D91819365
:1024300083E0E63EF807D1F7D3C061E070E087E6BD
:102440000E946D100E94C408CBC061E070E088E675
:102450000E946D1085E789838BE1EBECF3E0DE01F0
:10246000129601900D928A95E1F76CE1CE010196EA
:102470000E9460070E94DE0683E080939F0360E273
:1024800073E080E090E00E94311B80919F038430D4
:1024900009F0ADC08FE70E94FC040E940F058983FC
:1024A000853509F0A4C09CC061E070E08AE60E9416
:1024B0006D1089E6898361E0CE0101960E94600774
:1024C0000E94DE0683E080939F0360E273E080E079
:1024D00090E00E94311B80919F03843009F087C0F7
:1024E0008FE70E94FC040E940F0589838E010E5F16
:1024F0001F4F7E01EDE1EE0EF11C0E940F05F80169
:1025000081938F01EE15FF05C1F78BE1FE01329635
:10251000ABECB3E001900D928A95E1F789818934A3
:1025200009F065C05DC061E070E08BE60E946D104F
:10253000F8018081809300040E94CD0851C061E0C1
:1025400070E08CE60E946D10F0E2EF16F10461F489
:1025500087E6898380E2F801DE01129601900D92F0
:102560008A95E1F761E203C087E4898361E0CE01E7
:1025700001960E9460070E94DE0683E080939F031D
:102580006CE474E080E090E00E94311B80919F0336
:10259000843069F58FE70E94FC040E940F058734A0
:1025A00031F51EC061E070E08DE60E946D1089E19A
:1025B000E816F104E1F4D801E6EEF3E08D918193A1
:1025C00083E0EF3FF807D1F70BC061E070E08EE6E3
:1025D0000E946D10F80180818093FF030E94AE0875
:1025E00081E006C061E070E08AEC0E946D1080E03E
:1025F0000E944E100E948810A196E6E00C943E26A0
:10260000A0E0B0E0E6E0F3E10C942026CAE5D2E0D9
:1026100014E606E035E0F32E44E0E42E53E0D52E38
:1026200062E0C62E8AE094E00E947B1C892B09F4AC
:102630009BC08AE094E00E949F1C282F8093C502D3
:102640004091C40250E04730510560F7FA01EA5A60
:10265000FF4F0C944D26853B29F781E08093C402FF
:10266000E1CF823609F07DC0C092C402DBCF8093F7
:10267000C3028093C202D092C402D4CF9C013327FC
:102680003093C1022093C0029091C2029827909388
:10269000C202E092C402C6CF382F22274091C00266
:1026A0005091C102242B352B3093C1022093C002DC
:1026B0009091C20298279093C202F092C4022536EC
:1026C000310508F4AFCF61E070E08CEC0E946D1032
:1026D00081E00E944E100E94881043C02091BE02EB
:1026E0003091BF02F901E65AFD4F80839091C202FA
:1026F00098279093C202C90101969093BF028093DC
:10270000BE022091C0023091C1028217930708F4E3
:1027100089CF0093C40286CF8091C20282130BC07E
:102720006091BE027091BF024AE552E08091C302FF
:102730000E948F100DC062E070E08BEC0E946D1063
:102740008091C3020E944E10809196030E944E1009
:10275000FE01812F11928A95E9F71092BF02109223
:10276000BE021092C4025ECFCDB7DEB7E8E00C9493
:102770003C2681E08093970380919703882349F05A
:102780008AE094E00E947B1C892BB1F30E94001325
:10279000F3CF0895AAE2B0E0E0EDF3E10C941E2639
:1027A0000E94021B6B017C0181E00E9403068AE00B
:1027B00094E00E947B1C892B29F08AE094E00E941F
:1027C0009F1CF5CF5F9811E072E6B72EE9E2AE2EBE
:1027D00003E00E94021B6C197D098E099F09693C68
:1027E000710581059105D0F11123C1F10E94021BF1
:1027F0006B017C01469A80ED97E00E94FF02B9824E
:10280000E2EAF3E0DE0112968A2D01900D928A959C
:10281000E1F76AE2CE0101960E946007469880E0E7
:1028200090E00E94FF0200939F030E94DE0662E395
:1028300070E080E090E00E94311B80919F03843023
:1028400061F400939F038FE70E94FC040E940F0530
:1028500011E0823419F410E001C011E082E10E941D
:10286000521C892B81F411E00EC05F9A469A8AE0CF
:1028700094E00E949F1C8D309105A9F05CF40A97AA
:1028800091F05F9846988AE094E00E947B1C892B27
:1028900061F79FCF8332910569F08234910589F702
:1028A0000E94B913EECF66ED70E08AE094E00E94DA
:1028B000041EE7CF0E94DE0DE4CF8F929F92AF926D
:1028C000BF92CF92DF92EF92FF921F93CF93DF934D
:1028D00082E10E94521C892B09F089C068EC70E0EB
:1028E00080E090E00E94311B80E090E00E94FF02B7
:1028F0000E94021B4B015C016B017C0180ECC80E45
:1029000082E1D81EE11CF11C0E94021B6C157D05A2
:102910008E059F0530F482E10E94521C892BA1F3A1
:1029200064C082E10E94521C892B09F05EC080EDD8
:1029300097E00E94FF020E94021B6B017C01D0E025
:10294000C1E088E4880E86E2981EA11CB11C11E04B
:1029500082E10E94521C892B21F58C149D04AE0447
:10296000BF0430F480ED97E00E94FF02D1E0F0CF89
:102970000E94021B6C197D098E099F09693C710533
:102980008105910528F30E94021B6B017C01C12780
:1029900019F080ED97E002C080E090E00E94FF0215
:1029A000D7CF80E090E00E94FF02DD23B9F0809154
:1029B000FF0390E0019665E070E00E94C1258093DE
:1029C000FF030E94AE080E940E0B0E94CD0864EF28
:1029D00071E080E090E00E94311B09C080E00E941D
:1029E0004F020E942B090E94C4080E94CA13DF9163
:1029F000CF911F91FF90EF90DF90CF90BF90AF905D
:102A00009F908F900895CF92DF92EF92FF9280E097
:102A10000E945C030E94200361E086E00E94E61BA6
:102A200061E085E00E94E61B60E082E10E94E61B17
:102A300060E082E00E94E61B61E082E00E941F1CD1
:102A400060E083E00E94E61B61E083E00E941F1CBF
:102A500060E084E00E94E61B61E084E00E941F1CAD
:102A60000E94F30260E070E08AE094E00E94711D31
:102A70000E940E0B0E94CD080E94F30A8FEF8093F4
:102A80003A030E942C0378940E94021B6B017C0184
:102A900080913A038F3F59F40E94021B6C197D0903
:102AA0008E099F09603D77408105910588F380ED8F
:102AB00097E00E94FF0261E082E10E941F1C5F9A82
:102AC0008AE094E00E947B1C892B29F08AE094E044
:102AD0000E949F1CF5CF6EEE71E08AE094E00E94A8
:102AE000E51D86E893E00E94B50765E072E08AE0A4
:102AF00094E00E94E51D4AE050E066E070E08AE064
:102B000094E00E94AC1E62E370E080E090E00E94DE
:102B1000311B8AE094E00E947B1C04970CF18AE050
:102B200094E00E949F1C82349105D1F48AE094E0E5
:102B30000E949F1C8E34910599F48AE094E00E94D3
:102B40009F1C8434910561F48AE094E00E949F1CEC
:102B5000819731F480E090E00E94FF020E94CA1346
:102B60004091A3035091A4036091A5037091A60323
:102B7000DB01CA010197A109B1090497A105B105BB
:102B800068F440933903433029F440EA56E861E0A1
:102B900070E004C040E052EC61E070E08CE594E04D
:102BA0000E9441200E945D145F9880E090E00E94A6
:102BB000FF020E94F30A109259038091EB0383FFF6
:102BC00011C08091B703882351F08091BE03882300
:102BD00031F08091C503882311F087E001C085E0C2
:102BE0008093590380E00E94030680915A030E945B
:102BF00037050E94DE061092CF021092CE0210928C
:102C0000CD02F12C809100048F15B0F062E370E0EA
:102C100080E090E00E94311B80ED97E00E94FF026F
:102C200062E370E080E090E00E94311B80E090E081
:102C30000E94FF02F394E6CF8091CA0384FF08C08C
:102C4000982F987181E0983109F080E00E94E708A0
:102C50008FE00E945C03FF90EF90DF90CF9008958B
:102C6000EF92FF920F931F93CF93DF938C016EE748
:102C700070E08CE594E00E94C901E801F12CF0E2DB
:102C8000EF2E8E0188818D57823048F46DE770E019
:102C90008CE594E00E94C90188818E258883219665
:102CA000F80160818CE594E00E94531FF394F9E0F1
:102CB000FF12E7CF6EE770E08CE594E00E94C90157
:102CC000CDB7DEB7E6E00C943E26A9E0B0E0EBE637
:102CD000F6E10C94262690915B0391110EC09EEFB5
:102CE00099838A836B8350E0559547954C832D8358
:102CF000198618861F821E822EC040916003842F81
:102D000090E0B4E095958795BA95E1F7242F2F7060
:102D100030E08217930719F18DEF89831B82FE0142
:102D2000349650E0842F90E0A4E095958795AA957D
:102D3000E1F7242F2F7030E08217930749F0DC0170
:102D4000AF59BC4F8C918193405F5F5F563051F714
:102D5000409360035A83CE0101960E943016809101
:102D60005B0390E0019666E070E00E94C1258093CD
:102D70005B032996E2E00C944226A0E0B0E0E3EC8D
:102D8000F6E10C941F266C016EE770E08CE594E090
:102D90000E94C9018601E12CF12CC0E0D0E030E2B4
:102DA000B32EF801608183E8860F823078F46DE7F6
:102DB00070E08CE594E00E94C901F80160816B2508
:102DC00070E08CE594E00E94C90104C08CE594E0B9
:102DD0000E94531FE114F10459F0F80180819E0113
:102DE000280F311DC901C92FDD27C80FD91FDD27C5
:102DF0003FEFE31AF30A89E0E816F10459F028E0FE
:102E0000E216F10421F48C2F8095F60180870F5F84
:102E10001F4FC7CFCDB7DEB7E9E00C943B26A9E042
:102E2000B0E0E5E1F7E10C942626E82F362F8091FB
:102E30005B0390E0019664E270E00E94C1258093FC
:102E40005B0358E9598350E15A83813089F048F097
:102E50008230B9F08330D9F48B8381EF8C833D834A
:102E600019C085E08B8381EF8C832F5F2D8312C087
:102E70008B8381EF8C8384E6489FA00111245D83BE
:102E800009C084E08B8381EF8C83ED8303C00E94B3
:102E9000240904C0CE0101960E94BD162996E2E0E5
:102EA0000C944226A2E0B0E0E8E5F7E10C941B2682
:102EB000182F762E2A8349830E940E1B6B017C01FA
:102EC0008091710380905C0390905D03A0905E03FD
:102ED000B0905F032A8149818823C1F0D701C601E0
:102EE00088199909AA09BB094C015D0191EE89165F
:102EF0009EE29906A104B10420F1241708F4422FA0
:102F0000202F672D812F0E940F1713C0D701C601F4
:102F100088199909AA09BB094C015D0191E3891639
:102F200095E79906A104B10460F0672D812F0E94F6
:102F30006516C0925C03D0925D03E0925E03F0924E
:102F40005F032296EDE00C943726A2E2B0E0EBEAB4
:102F5000F7E10C941C268CE00E941E0581110DC027
:102F60006DE072E08AE094E00E94161E5F9A80E0B5
:102F70000E9403060E94DE065F988CE594E00E94A2
:102F8000F91E892B01F18CE594E00E94261F909197
:102F90003903992319F00E944A0BEFCF4091CE02DA
:102FA00050E09A012F5F3F4F2F7133276091CF027E
:102FB00070E02617370709F3FA01E752FD4F8083C7
:102FC0002093CE02DACF80913903811106C080911F
:102FD0009F03843009F094C00DC08AE094E00E9401
:102FE0007B1C892BA1F38AE094E00E949F1C0E9425
:102FF0004A0BF3CF0E940E1B6115710581059105E7
:1030000049F060934B0370934C0380934D0390936E
:103010004E030CC081E090E0A0E0B0E080934B0351
:1030200090934C03A0934D03B0934E0380913D03C6
:1030300090913E03816090933E0380933D0383E033
:1030400080939F038FE70E94FC0409EF12E00E9427
:103050000F05F80181938F01F3E002301F07B9F7E4
:10306000209102038091F902982F922796FF3BC08E
:1030700090E4922790930203982F98739833F1F479
:1030800010E0212F30E08091F902877090E08217E4
:1030900093074CF11F5F2091CA03812F90E0FC0140
:1030A000E750FD4F24FF04C080810E940609E9CF4C
:1030B00060818CE594E00E94531FE3CF8F7399F4F5
:1030C0008091FA02809346038091FB02809344032F
:1030D0008091FC02809343038091FF0290E09093E3
:1030E0003C0380933B038091CD02813019F482E050
:1030F0008093CD028091CD02833011F41092CD02E5
:103100000E940E1B6B017C0180913F039091400354
:10311000A0914103B09142030097A105B105C9F008
:10312000A7019601281B390B4A0B5B0BDA01C90179
:10313000883B9B40A105B10560F00E944D0580933E
:10314000450310923F0310924003109241031092E6
:10315000420380914F0390915003A0915103B0918D
:10316000520346015701881A990AAA0ABB0A82EA41
:1031700093E00E94780386169706A806B90608F41D
:10318000B1C0C0924F03D0925003E0925103F0922D
:1031900052030E94C00180913A038830A0F08091D0
:1031A000EB039091EC03A091ED03B091EE035CE191
:1031B000B695A795979587955A95D1F7892B8A2B20
:1031C0008B2B09F0C4C180913A038F5F80933A033F
:1031D00080914B0390914C03A0914D03B0914E030D
:1031E0000097A105B105F1F0C81AD90AEA0AFB0A4D
:1031F00082EA93E00E9478036C157D058E059F0599
:1032000008F01BC18091EB0384FD04C080ED97E0C2
:103210000E94FF0210924B0310924C0310924D0338
:1032200010924E0390910203907C90930203509170
:10323000CE028091CF022091CD02581709F41AC115
:10324000223009F017C1905890930203E091CA030D
:10325000E770F0E0E45EFD4F6081693008F0F2C095
:10326000615040E04613F0C08093CF0287E3840FA3
:1032700090910203892B809302034093D00283E054
:103280008093CD02469A1091AF038091590381112A
:103290003EC18091EB0382FD46C1812F0E94FE0555
:1032A00080915A030E943705E091CA03E770F0E06D
:1032B000E45EFD4F608182E093E00E9419078091F7
:1032C000EB0382FD39C1E0915A03EF5FE0935A03AB
:1032D000E83109F439C1F0E0EE55FC4F87858823C9
:1032E00009F432C10E948807813069F58091CA03D0
:1032F000887149F180913D0390913E03880F991F99
:1033000090933E0380933D0383E080939F030E944C
:10331000DE060E940E1B60933F0370934003809370
:10332000410390934203672B682B692B61F481E082
:1033300090E0A0E0B0E080933F0390934003A0931F
:103340004103B09342038091CA0384FF2BC0809154
:103350004B0390914C03A0914D03B0914E03892BE8
:103360008A2B8B2BF9F080913D0390913E038E7F49
:103370000E94AE04182F60913B03809146030E9487
:10338000400B482F612F8091450349A30E94400BB9
:1033900000910004282F49A16091430380914403C8
:1033A0000E9452174698809157038130C1F018F05F
:1033B0008230B1F1D9C082E10E94521C892B09F000
:1033C000D3C081E0809357030E94021B6093530394
:1033D000709354038093550390935603C5C082E1C4
:1033E0000E94521C892B31F50E94021BC09053038E
:1033F000D0905403E0905503F09056036C197D096A
:103400008E099F09693E73408105910508F4ACC09F
:1034100082E08093570380ED97E00E94FF02A4C0F2
:1034200082E10E94521C892B09F49EC080E090E04A
:103430000E94FF021092570397C080E090E00E9424
:10344000FF02F0CE68E00DCF851709F40DCF4F5F76
:10345000242F30E090E0F901EE5FFC4FDC01A75231
:10346000BD4F7C917083F901E053FD4F708301964D
:103470008F71F8CE2430B1F42091D00281ED92E02A
:10348000A3E0B3E0FC013E2F381B321718F4319152
:103490003D93F9CF87E3820F90910203892B8093AC
:1034A0000203EDCE80915703823051F491609093E6
:1034B00002035F9A8E010F5F1F4FF12CB80110C0FD
:1034C0005F988091CD02811103C081E08093CD028D
:1034D0008091CD02833071F784E08093CD02EACFF2
:1034E0008F2D69A37AA30E94690DF80181939193AE
:1034F0008F01F39469A17AA1F0E1FF12F1CF8091DD
:10350000CA0343E053E087700E94FD03BBCE112342
:1035100009F4BFCE9091580321E0290F209358035E
:103520009813B7CE1DC082E00E94521C892B09F06F
:10353000B4CE5F9A17E0B1CE82E00E94521C892B74
:1035400009F0C1CE5F98BFCE10925A03CBCE8091C6
:103550003A03883009F45F9A89E080933A03C2CE37
:1035600010925803115095CEA296ECE00C94382698
:103570001F920F920FB60F9211242F933F938F93A8
:103580009F93AF93BF938091020490910304A09105
:103590000404B09105043091010423E0230F2D377A
:1035A00020F40196A11DB11D05C026E8230F029647
:1035B000A11DB11D20930104809302049093030484
:1035C000A0930404B093050480910604909107042D
:1035D000A0910804B09109040196A11DB11D80932A
:1035E000060490930704A0930804B0930904BF91C4
:1035F000AF919F918F913F912F910F900FBE0F90A0
:103600001F9018952FB7F8946091020470910304ED
:1036100080910404909105042FBF08953FB7F8945A
:103620008091060490910704A0910804B0910904C8
:1036300026B5A89B05C02F3F19F00196A11DB11D0D
:103640003FBF6627782F892F9A2F620F711D811D2A
:10365000911D42E0660F771F881F991F4A95D1F789
:103660000895CF92DF92EF92FF92CF93DF936B0199
:103670007C010E940E1BEB01C114D104E104F10492
:1036800079F00E940E1B6C1B7D0B683E7340A0F30B
:1036900081E0C81AD108E108F108C851DC4FECCF2D
:1036A000DF91CF91FF90EF90DF90CF9008957894C5
:1036B00084B5826084BD84B5816084BD85B5826037
:1036C00085BD85B5816085BDEEE6F0E080818160D5
:1036D0008083E1E8F0E010828081826080838081D5
:1036E00081608083E0E8F0E0808181608083E1E9AF
:1036F000F0E0808182608083808181608083E0E966
:10370000F0E0808181608083E1ECF0E08081846082
:103710008083808182608083808181608083E3EC0C
:10372000F0E0808181608083E0ECF0E08081826065
:103730008083E2ECF0E0808181608083EAE7F0E062
:1037400080818460808380818260808380818160C9
:103750008083808180688083089590E0FC013197A8
:10376000EE30F10590F5E35AFF4F0C944D26809111
:1037700080008F7703C0809180008F7D80938000D0
:10378000089584B58F7702C084B58F7D84BD089578
:10379000809190008F7707C0809190008F7D03C04B
:1037A00080919000877F8093900008958091C00061
:1037B0008F7703C08091C0008F7D8093C0000895F3
:1037C0008091C200877F8093C2000895CF93DF93DA
:1037D00090E0FC01E75EFE4F2491FC01E95CFE4FA6
:1037E0008491882349F190E0880F991FFC01EF58DC
:1037F000FE4FA591B4918D599E4FFC01C591D49176
:103800009FB7611108C0F8948C91209582238C9306
:10381000888182230AC0623051F4F8948C91322F4F
:10382000309583238C938881822B888304C0F894FD
:103830008C91822B8C939FBFDF91CF910895A1E053
:10384000B0E0E5E2FCE10C942426282F30E0F901F9
:10385000E550FF4F8491F901E75EFE4F1491F901A5
:10386000E95CFE4F04910023C9F0882321F06983AD
:103870000E94AD1B6981E02FF0E0EE0FFF1FED59B4
:10388000FE4FA591B4919FB7F8948C91611103C03C
:103890001095812301C0812B8C939FBF2196E4E07A
:1038A0000C944026CF93DF93282F30E0F901E550A8
:1038B000FF4F8491F901E75EFE4FD491F901E95C75
:1038C000FE4FC491CC2391F081110E94AD1BEC2FCF
:1038D000F0E0EE0FFF1FEB5AFE4FA591B4912C9133
:1038E0002D2381E090E021F480E002C080E090E0B0
:1038F000DF91CF91089580915804909159042091BF
:103900005A0430915B04821B930B8F73992708959F
:10391000209158043091590480915A0490915B048D
:103920002817390749F0E0915A04F0915B04E85EEA
:10393000FB4F808190E008958FEF9FEF08952091D5
:1039400058043091590480915A0490915B042817CF
:103950003907A9F0E0915A04F0915B04E85EFB4F4F
:10396000808120915A0430915B042F5F3F4F2F7369
:10397000332730935B0420935A0490E008958FEF2F
:103980009FEF0895CF93DF93C0915804D0915904CD
:103990002196CF73DD2780915A0490915B04C8175C
:1039A000D90799F082E00E9477218F3F2FEF92078D
:1039B00061F0E0915804F0915904E85EFB4F808378
:1039C000D0935904C0935804DFCFDF91CF9108956D
:1039D00083E00E94C2230895A1E0B0E0E2EFFCE1A1
:1039E0000C9424268C0169838091A401882359F0CA
:1039F00041E050E0BE016F5F7F4F83E00E94AA214B
:103A0000181619063CF081E090E0F8019383828358
:103A100080E090E02196E4E00C944026FC012081B7
:103A20002E5F208342E450E06FE771E080E80E945F
:103A30002A220895FC0181819081913A59F48132C2
:103A400009F04BC047E050E06DE971E080E00E9472
:103A50002A2245C0913209F040C0803239F467E033
:103A600070E08DE991E00E946E2239C0823209F047
:103A700034C082818093A40180919D0190919E0128
:103A8000A0919F01B091A001803B9440A105B10598
:103A900031F58091A40180FD12C087E797E79093EC
:103AA0000108809300082BE088E190E00FB6F894BD
:103AB000A895809360000FBE2093600010C088E13D
:103AC0000FB6F89480936000109260000FBEA89526
:103AD000109201081092000802C080E0089581E071
:103AE0000895089510920D0410920C0488EE93E04E
:103AF000A0E0B0E080930E0490930F04A093100414
:103B0000B09311048EE292E090930B0480930A0428
:103B10000895A0E0B0E0EFE8FDE10C9420266C01F0
:103B20007A01EB01E60EF71E00E010E0CE15DF058E
:103B300061F06991D601ED91FC910190F081E02D49
:103B4000C6010995080F191FF1CFC801CDB7DEB71F
:103B5000E8E00C943C266115710589F0DB010D90BD
:103B60000020E9F7AD0141505109461B570BDC011C
:103B7000ED91FC910280F381E02D0995089580E09C
:103B800090E00895EF92FF920F931F93CF93DF93EE
:103B90008C01FB01C0E0D0E064917F018FEFE81A57
:103BA000F80A662361F0D801ED91FC910190F08153
:103BB000E02DC8010995C80FD91FF701EDCFCE013F
:103BC000CDB7DEB7E6E00C943E260E94AB1D08950B
:103BD000DC01ED91FC910190F081E02D09950895B3
:103BE0000F931F93CF93DF93EC016DE00E94E81DCC
:103BF0008C016AE0CE010E94E81D800F911FDF91C9
:103C0000CF911F910F9108950F931F93CF93DF933F
:103C1000EC010E94C21D8C01CE010E94F01D800F9C
:103C2000911FDF91CF911F910F9108950F931F93D3
:103C3000CF93DF93EC010E94AB1D8C01CE010E945B
:103C4000F01D800F911FDF91CF911F910F9108956B
:103C50000F931F93CF93DF93EC010E94E81D8C011B
:103C6000CE010E94F01D800F911FDF91CF911F9117
:103C70000F910895A1E2B0E0E0E4FEE10C941C266F
:103C80007C01C42EE52FCB01D22E19A221E02D15E7
:103C900010F02AE0D22E8E010F5D1F4F8D2C912C3B
:103CA000A12CB12C6C2D7E2FA50194010E94D5254D
:103CB0008C2DD29E80191124015011098A3010F4E4
:103CC000805D01C0895CF8018083211531054105C3
:103CD000510521F0C22EE32FCA01E4CFB801C7017C
:103CE0000E94AB1DA196ECE00C943826A0E0B0E059
:103CF000ECE7FEE10C942026EC016A017B01211522
:103D0000310541F4E881F9810190F081E02D642FC3
:103D100009951DC02A303105A9F477FF12C06DE264
:103D20000E94E81D8C0144275527BA014C195D09F2
:103D30006E097F092AE0CE010E943A1E800F911F72
:103D400006C02AE0B701A601CE010E943A1ECDB7F7
:103D5000DEB7E8E00C943C260F931F93CF93DF93DC
:103D6000EC019A01AB01662757FD6095762F0E9402
:103D7000761E8C01CE010E94F01D800F911FDF91F5
:103D8000CF911F910F9108952115310549F4DC0160
:103D9000ED91FC910190F081E02D642F099508953B
:103DA0000E943A1E08959A01462F50E060E070E0AC
:103DB0000E94C41E08959A01AB0160E070E00E9469
:103DC000C41E08950F931F93CF93DF93EC019A01C4
:103DD000462F50E060E070E00E94C41E8C01CE01CE
:103DE0000E94F01D800F911FDF91CF911F910F91C5
:103DF0000895FC0124853585F901E05CFF4F808141
:103E00009181F901EE5BFF4F20813181821B930B81
:103E10008F7399270895FC0184859585FC01E05CEA
:103E2000FF4F40815181FC01EE5BFF4F20813181CA
:103E30004217530741F00190F081E02DE80FF91F80
:103E4000808190E008958FEF9FEF0895FC018485B5
:103E50009585FC01E05CFF4F40815181FC01EE5BE8
:103E6000FF4F208131814217530779F0A081B18142
:103E7000A80FB91F8C91208131812F5F3F4F2F7385
:103E800033273183208390E008958FEF9FEF0895CB
:103E9000FC0181A1882329F0A489B5898C9186FF32
:103EA000FBCF11A20895CF93DF93FC0126853785C0
:103EB000D901A05CBF4F8D919C91119701968F7392
:103EC0009927E901CE5BDF4F488159818417950717
:103ED000D9F30D90BC91A02DA20FB31F6C93A685B2
:103EE000B785A05CBF4F11969C938E93A689B78926
:103EF0002C9181E090E0078C02C0880F991F0A94F2
:103F0000E2F7282B2C9381E081A30488F589E02D2A
:103F100080818064808381E090E0DF91CF9108957B
:103F200008951F920F920FB60F9211242F933F9373
:103F30004F938F939F93EF93FF938091C80082FDDF
:103F40001CC04091CE00809102059091030501961E
:103F50008F739927209104053091050582179307E7
:103F600071F0E0910205F0910305EE53FB4F4083A1
:103F7000909303058093020502C08091CE00FF91CB
:103F8000EF919F918F914F913F912F910F900FBE85
:103F90000F901F9018958CE594E00E94F91E892BD4
:103FA00011F00E94901F08951F920F920FB60F926A
:103FB00011242F933F938F939F93EF93FF9320911F
:103FC000BE043091BF048091C0049091C1042817B1
:103FD000390731F48091C9008F7D8093C90014C0E6
:103FE000E091C004F091C104E258FB4F2081809120
:103FF000C0049091C10401968F7399279093C104D6
:104000008093C0042093CE00FF91EF919F918F91F8
:104010003F912F910F900FBE0F901F901895A0E029
:10402000B0E0E5E1F0E20C941C26FC011382128260
:1040300088EE93E0A0E0B0E084839583A683B78305
:1040400080E492E0918380837587648757874687F1
:10405000318B208B138B028BF58AE48AD78AC68A30
:10406000B18EA08E938E828E8F85848F8889858F66
:104070008989868F8A89878F8B8980A3ECE00C944D
:104080003826CF92DF92EF92FF92CF93DF93EC012D
:104090006A017B01411581EE580761057105F9F050
:1040A000EC89FD8981E090E008A002C0880F991F8B
:1040B0000A94E2F7808360E079E08DE390E0A70165
:1040C00096010E94D5252150310941095109569583
:1040D000479537952795211580E1380798F0EC89A9
:1040E000FD89108260E874E88EE190E0A7019601F6
:1040F0000E94D5252150310941095109569547950E
:1041000037952795E889F9893083EA89FB892083E7
:1041100019A2EE89FF89408181E090E09C010C8C1E
:1041200002C0220F331F0A94E2F7422B4083EE892C
:10413000FF8940819C010D8C02C0220F331F0A941D
:10414000E2F7422B4083EE89FF8940819C010E8C6F
:1041500002C0220F331F0A94E2F7422B4083EE89FC
:10416000FF8920810F8C02C0880F991F0A94E2F703
:10417000809582238083DF91CF91FF90EF90DF9035
:10418000CF9008958F929F92AF92BF92CF92DF927D
:10419000EF92FF920F931F9381E08F9385E08F93AF
:1041A00087E08F9383E08F9384E08F93EEEC8E2EE5
:1041B000912CFAECAF2EB12CA9ECCA2ED12CB8EC74
:1041C000EB2EF12C0CEC10E02DEC30E04EE754E03F
:1041D00062EC74E08CE594E00E940F200F900F9049
:1041E0000F900F900F901F910F91FF90EF90DF9025
:1041F000CF90BF90AF909F908F9008950E94571BD3
:1042000086E095E00E94CC230E940315CBECDFE111
:104210000E94A5172097E1F30E94CB1FF9CF6150B0
:1042200030F02091F100FC0120830196F8CF28980E
:1042300084E680930D0508952FB7FC012083F89440
:1042400067706093E9000895A1E0B0E0EAE2F1E26E
:104250000C942626682FCE0101960E941C21809185
:10426000F20099819FBF2196E2E00C944226A2E0E1
:10427000B0E0EDE3F1E20C942326F62E8A01909152
:104280000C05992311F057FF03C08FEF9FEF2BC050
:10429000682FCE0101967A830E941C218091F20042
:1042A00090E0A8017A81801791070CF4AC01EF2D02
:1042B000F72FF40E84E6FE1639F0289880930D054A
:1042C0009091F1009193F7CF4115510521F0809124
:1042D000F200882321F089818FBFCA0104C08BE6D8
:1042E0008093E800F8CF2296E5E00C943F26A1E009
:1042F000B0E0EDE7F1E20C94262641E050E0BE018B
:104300006F5F7F4F0E943721019719F4898190E0F8
:1043100002C08FEF9FEF2196E2E00C944226A1E0CD
:10432000B0E0E5E9F1E20C942626682FCE01019673
:104330000E941C219091E800892F807295FF04C093
:104340009091F20080E4891B99819FBF2196E2E061
:104350000C944226A1E0B0E0E0EBF1E20C941826C8
:10436000582E7B01A42E952E80910C05882369F090
:10437000042F152F8AEFB82E852D8072782E9AE3A0
:10438000892E852D8074682E11C08FEF9FEF53C04A
:10439000852D0E948F21482E81110CC0BA94A9F35B
:1043A00061E070E080E090E00E94311B0115110592
:1043B00079F737C0282F30E0021713070CF4402E8E
:1043C000C42CD12C0C191D09652DCE0101960E941B
:1043D0001C21772039F04A948FEF4816B1F01092E3
:1043E000F100F9CFF701842D57FE07C0815058F036
:1043F00094919093F1003196F9CF815020F09191F2
:104400009093F100FACFEC0CFD1C8091E80085FF41
:104410000FC00115110511F461100AC089818FBF09
:10442000C5CF5D9884E680930E058A2D992D03C033
:104430008092E800F3CF2196E0E10C9434261092AC
:10444000E90010920B0510920A05909309058093DC
:1044500008050895CF93DF93FB0120E030E0DEEF05
:1044600024173507A1F187FF02C0C49101C0C081A4
:10447000A0910A05B0910B0560910805709109059E
:10448000A617B707B4F49091E8009570E1F3909106
:10449000E80092FD1EC0C093F10060910A05709182
:1044A0000B056F5F7F4F6F737727672B11F4D093E6
:1044B000E80060910A0570910B056F5F7F4F709364
:1044C0000B0560930A052F5F3F4F3196C9CFC90195
:1044D00002C08FEF9FEFDF91CF910895A1E0B0E090
:1044E000E4E7F2E20C942526162F2091E80022FF43
:1044F000FCCF612F79830E940F218BEF8093E8001E
:10450000812F7981972F2196E3E00C944126A1E039
:10451000B0E0EDE8F2E20C9426261982CE01019675
:104520000E940E1DCE0101960E946624898190E0B2
:104530002196E2E00C9442261F920F920FB60F9242
:104540001124EF92FF920F931F932F933F934F935A
:104550005F936F937F938F939F93AF93BF93EF93EB
:10456000FF93CF93DF93CDB7DEB76297DEBFCDBFAA
:104570001092E9008091E80083FFE7C068E0CE0177
:104580000A960E940F2182EF8093E8009A8597FF98
:1045900005C08091E80080FFFCCF03C08EEF8093C0
:1045A000E800892F807609F0B5C08B85811105C0A0
:1045B0001092F1001092F100C1C0282F2D7F213000
:1045C00009F4BCC0853049F48091E80080FFFCCF3D
:1045D0008C8580688093E300B1C0863009F072C09A
:1045E0002D85E888F988223071F580E090E02A8BEB
:1045F0000E941F220E94872299E08E010F5F1F4FA9
:10460000F801392F11923A95E9F799832A892A837B
:1046100091E09E8390E898879AEF998720910A0508
:1046200030910B05275F3F4F3C832B838D83C70160
:104630000E941F2249E050E0B80180E00E942A2237
:104640000E9487227BC0C7012A8B0E941F222A89D1
:10465000223241F482E290E00E947224892B09F018
:104660006DC070C0213069F488899989089711F468
:104670002093070580910705882389F066EC71E097
:1046800016C0233009F05EC08C85882359F0823033
:1046900061F0813009F056C06AEE71E008C068ED43
:1046A00071E005C064E272E002C062E072E0611590
:1046B000710509F447C0FB01449150E080E80E9475
:1046C0002A223CC0873009F43DC0883021F481E0C3
:1046D0008093F10033C0893089F5937099F5E2EC4D
:1046E000F1E081E021E096E38093E9002093EB0084
:1046F00034913093EC009093ED008F5F31968530CC
:1047000099F78EE78093EA001092EA008C858093F7
:104710000C0514C0888999890E941F228E858111F9
:1047200005C0CE010A960E941A1D06C0823051F4BF
:10473000CE010A960E949424882321F08EEF809364
:10474000E80003C081E28093EB0062960FB6F89414
:10475000DEBF0FBECDBFDF91CF91FF91EF91BF9133
:10476000AF919F918F917F916F915F914F913F9109
:104770002F911F910F91FF90EF900F900FBE0F9010
:104780001F9018958093E9008091F200882319F01A
:104790008AE38093E800089510920C0581E08093ED
:1047A000D70080EA8093D80082E189BD09B400FE79
:1047B000FDCF61E070E080E090E00E94311B80E975
:1047C0008093D8008CE08093E2001092E000559A2C
:1047D000209A08951F920F920FB60F9211242F93D3
:1047E0003F934F935F936F937F938F939F93AF9379
:1047F000BF93EF93FF938091E1001092E10083FF5C
:104800000FC01092E90091E09093EB001092EC0041
:1048100092E39093ED0010920C0598E09093F000D5
:1048200082FF26C083E00E94C22382E00E942421EE
:10483000882321F08AE094E00E94C21C80910E053A
:10484000882339F080910E05815080930E058823CE
:1048500069F080910D05882359F080910D058150F4
:1048600080930D05811104C0289A02C05D9AF1CF92
:10487000FF91EF91BF91AF919F918F917F916F9138
:104880005F914F913F912F910F900FBE0F901F900E
:104890001895FF920F931F93CF93DF93EC01F62EA1
:1048A000E881F9810480F581E02D09958C01E8818A
:1048B000F9810680F781E02D6F2DCE010995C801A1
:1048C0009927CDB7DEB7E5E00C943F26FC012081A7
:1048D0002F5F208349E150E068EA72E080E80E949F
:1048E0002A22089545E650E061EC72E080E80E94DB
:1048F0002A220895A1E0B0E0E0E8F4E20C94222638
:1049000089838B017A0141E050E0BE016F5F7F4FE8
:1049100084E00E94AA21A701B80184E40E94AA2190
:104920002196E6E00C943E26FC0191818081813A3B
:1049300031F481E0913091F0933089F411C08132EB
:1049400071F49B3021F482818093A60105C09A30D6
:1049500031F482818093A50181E00895089580E07B
:104960000895FC0110820895FC011382128220E553
:1049700032E031832083089548E050E082E00E94D5
:104980007A240895CF93DF93DC01683818F0E8E7C4
:10499000E60F25C0E62FF0E067FF11C0E058F109EF
:1049A00081E090E001C0880FEA95EAF714969C91A7
:1049B0001497982B14969C931497E0E010C0E85D30
:1049C000FD4FE491EE2309F440C0E7FF08C01496C0
:1049D0008C911497826014968C931497EF771696A7
:1049E0008C9116978E1741F117968C9117978E1709
:1049F00019F118968C9118978E17F1F019968C91E1
:104A000019978E17C9F01A968C911A978E17A1F0E4
:104A10001B968C911B978E1779F080E090E0ED014A
:104A2000C80FD91F2E81211102C0EE8305C0019647
:104A300086309105A1F709C0BD016C5F7F4FCD01A4
:104A40000E94BC2481E090E008C081E090E01396D1
:104A50009C938E93129780E090E0DF91CF91089520
:104A6000683818F0E8E7E60F25C0E62FF0E067FFAA
:104A700012C0E058F10921E030E001C0220FEA95B0
:104A8000EAF72095DC0114963C9114973223149692
:104A90003C93E0E00FC0E85DFD4FE491EE2329F187
:104AA000E7FF08C0DC0114962C9114972D7F149613
:104AB0002C93EF7720E030E0EE2351F0DC01A20FE1
:104AC000B31F16964C9116974E1302C016961C9261
:104AD0002F5F3F4F2630310579F7BC016C5F7F4F68
:104AE0000E94BC2481E090E0089580E090E0089569
:104AF000FC01168217821086118612861386148294
:104B0000BC016C5F7F4F0E94BC2408958BE195E04F
:104B10000E94B1248FE095E00E94B4240895A29FE2
:104B2000B001B39FC001A39F700D811D1124911D81
:104B3000B29F700D811D1124911D08950E948F2533
:104B4000A59F900DB49F900DA49F800D911D1124E1
:104B50000895B7FF0C949E250E949E25821B930BFF
:104B60000895DB018F939F930E949E25BF91AF9183
:104B7000A29F800D911DA39F900DB29F900D1124B7
:104B8000089597FB072E16F4009407D077FD09D0FF
:104B90000E94532607FC05D03EF4909581959F4FC7
:104BA0000895709561957F4F0895A1E21A2EAA1B72
:104BB000BB1BFD010DC0AA1FBB1FEE1FFF1FA217CD
:104BC000B307E407F50720F0A21BB30BE40BF50BCA
:104BD000661F771F881F991F1A9469F76095709553
:104BE000809590959B01AC01BD01CF010895052EE4
:104BF00097FB1EF400940E940E2657FD07D00E94DA
:104C0000D52507FC03D04EF40C940E265095409504
:104C1000309521953F4F4F4F5F4F08959095809568
:104C2000709561957F4F8F4F9F4F08952F923F92C0
:104C30004F925F926F927F928F929F92AF92BF92AC
:104C4000CF92DF92EF92FF920F931F93CF93DF9358
:104C5000CDB7DEB7CA1BDB0B0FB6F894DEBF0FBEB5
:104C6000CDBF09942A88398848885F846E847D8402
:104C70008C849B84AA84B984C884DF80EE80FD8004
:104C80000C811B81AA81B981CE0FD11D0FB6F8947A
:104C9000DEBF0FBECDBFED010895EE0FFF1F0590E3
:104CA000F491E02D0994AA1BBB1B51E107C0AA1F78
:104CB000BB1FA617B70710F0A61BB70B881F991FBD
:104CC0005A95A9F780959095BC01CD0108958F92D2
:104CD0009F92AF92BF92CF92DF92EF92FF92CF93CB
:104CE000DF93EC01688179818A819B81611571056F
:104CF0008105910521F464E279ED8BE597E02DE1E2
:104D000033EF41E050E00E94F72549015A019B0131
:104D1000AC01A7EAB1E40E949E256B017C01ACEED8
:104D2000B4EFA50194010E94AC25C60ED71EE81E63
:104D3000F91EF7FE06C081E0C81AD108E10880E834
:104D4000F80AC882D982EA82FB82C701B6019F773E
:104D5000DF91CF91FF90EF90DF90CF90BF90AF9019
:104D60009F908F9008950E946726089586E091E0B5
:104D70000E9467260895609306017093070180934F
:104D80000801909309010895F999FECF92BD81BD64
:104D9000F89A992780B50895262FF999FECF1FBA62
:104DA00092BD81BD20BD0FB6F894FA9AF99A0FBE54
:084DB00001960895F894FFCF6D
:104DB80000001C05200001000000FF0002000200A6
:104DC80002000200020002000200020002000200CB
:104DD8000200020002000200020002802500000515
:104DE800400AA1204EA50020244EA52C2330C01235
:104DF80000001A400AA1204EA5001B1E27522C2392
:104E0800308025000005400AA1204EA50020244E30
:104E1800A52C2330004B000006400AD0009D490015
:104E28007B289D492C233000E1000005400A4501FC
:104E3800D7DC03B81E0EBF00232E48E801008A40C5
:104E48000A6001555502AD1E20000023C800E1008C
:104E58000000000000010154582074696D656F75E9
:104E6800742100456E746572696E672061646170B3
:104E780074697665206368616E6E656C2073656C15
:104E8800656374696F6E2C207069636B696E673A2D
:104E9800007363616E6E6572206D6F6465004F709C
:104EA800656E4C52536E6720545820737461727447
:104EB800696E672000206F6E20485720006D6F6470
:104EC800756C65206C6F636B65643F0000070B0CA5
:104ED80010111500160A1322312900000000EC1CDD
:104EE800891D7B1C9F1C881CE81CC21C000000003C
:104EF800531F891DF91E261F0B1F481F00000000A5
:0A4F08004924891DC22430257825B4
:00000001FF
